:10000000010AA304C50C0200040061006600380C5C
:100010000600030C3300640C3500040C3600780035
:10002000E60CC101030634093806200958061909EF
:10003000100A580446071E0A460400084605000830
:1000400038041602E201270A290A2B0A2D0A26047F
:100050002F0A26052F0A06042F0A06052F0AF60284
:100060000008040C3600000804006100F3020008D8
:10007000030C33003805F5020008640C3500580500
:02008000000876
:021FFE00EE0FE4
:00000001FF
